:020000040800F2
:1000000000060020F50500081D350008D53400085D
:10001000FD340008D5340008F5340008F705000861
:10002000F7050008F7050008F70500080145000876
:10003000F7050008F7050008F7050008F7050008B0
:10004000F7050008F7050008F7050008F7050008A0
:10005000F7050008F7050008F15C00081D5D0008C1
:10006000495D0008755D0008A15D0008F7050008FE
:10007000F7050008F7050008F7050008F705000870
:10008000F7050008F7050008F705000885340008A3
:10009000AD34000899340008C1340008CD5D000873
:1000A000F7050008F7050008F7050008F705000840
:1000B000F7050008F7050008F7050008F705000830
:1000C000F7050008F7050008F7050008F705000820
:1000D000F7050008A55E0008F7050008F705000809
:1000E000315E0008F7050008F7050008F70500086D
:1000F000F7050008F7050008F7050008F7050008F0
:10010000F7050008F7050008CD5E0008F7050008B0
:10011000F7050008F7050008F7050008F7050008CF
:10012000F7050008F7050008F7050008F7050008BF
:10013000F7050008F7050008F7050008F7050008AF
:10014000F7050008F7050008F7050008F70500089F
:10015000F7050008F7050008F7050008F70500088F
:10016000F7050008F7050008F7050008F70500087F
:10017000F7050008F7050008F7050008F70500086F
:10018000F7050008F7050008F7050008B95E000844
:10019000F7050008F7050008F7050008F70500084F
:1001A000F7050008F7050008F7050008F70500083F
:1001B000F7050008F7050008F7050008F70500082F
:1001C000F7050008F7050008F7050008F70500081F
:1001D000F7050008F7050008F7050008F70500080F
:1001E000F7050008F7050008F7050008F7050008FF
:1001F000F7050008F7050008F7050008F7050008EF
:10020000F7050008F7050008F7050008F7050008DE
:10021000F7050008F7050008F7050008F7050008CE
:10022000F7050008F7050008F7050008F7050008BE
:10023000F7050008F7050008F7050008F7050008AE
:10024000F7050008F7050008F7050008F70500089E
:10025000F7050008F7050008F7050008F70500088E
:10026000F7050008F7050008F7050008F70500087E
:10027000F7050008F7050008F7050008F70500086E
:10028000F7050008F7050008F7050008F70500085E
:10029000F7050008F7050008F7050008F70500084E
:1002A000F7050008F7050008F7050008F70500083E
:1002B000F7050008F7050008F7050008F70500082E
:1002C000F7050008F7050008F7050008F70500081E
:1002D000F7050008F7050008F7050008F70500080E
:1002E000CD19000800000000000000000000000020
:1002F00053B94AB9002908BF00281CBF4FF0FF318D
:100300004FF0FF3000F074B9ADF1080C6DE904CE88
:1003100000F006F8DDF804E0DDE9022304B07047E0
:100320002DE9F047089D04468E46002B4DD18A42A8
:10033000944669D9B2FA82F252B101FA02F3C2F1DB
:10034000200120FA01F10CFA02FC41EA030E94406C
:100350004FEA1C48210CBEFBF8F61FFA8CF708FB8D
:1003600016E341EA034306FB07F199420AD91CEB65
:10037000030306F1FF3080F01F81994240F21C8197
:10038000023E63445B1AA4B2B3FBF8F008FB1033DF
:1003900044EA034400FB07F7A7420AD91CEB040414
:1003A00000F1FF3380F00A81A74240F207816444E4
:1003B000023840EA0640E41B00261DB1D440002369
:1003C000C5E900433146BDE8F0878B4209D9002DCD
:1003D00000F0EF800026C5E9000130463146BDE857
:1003E000F087B3FA83F6002E4AD18B4202D38242C1
:1003F00000F2F980841A61EB030301209E46002D70
:10040000E0D0C5E9004EDDE702B9FFDEB2FA82F2C4
:10041000002A40F09280A1EB0C014FEA1C471FFA22
:100420008CFE0126200CB1FBF7F307FB131140EA09
:1004300001410EFB03F0884208D91CEB010103F1D6
:10044000FF3802D2884200F2CB804346091AA4B298
:10045000B1FBF7F007FB101144EA01440EFB00FE6C
:10046000A64508D91CEB040400F1FF3102D2A645D1
:1004700000F2BB800846A4EB0E0440EA03409CE770
:10048000C6F12007B34022FA07FC4CEA030C20FA1D
:1004900007F401FA06F31C43F9404FEA1C4900FA3D
:1004A00006F3B1FBF9F8200C1FFA8CFE09FB1811BA
:1004B00040EA014108FB0EF0884202FA06F20BD92D
:1004C0001CEB010108F1FF3A80F08880884240F27D
:1004D0008580A8F102086144091AA4B2B1FBF9F0C1
:1004E00009FB101144EA014100FB0EFE8E4508D9BC
:1004F0001CEB010100F1FF346CD28E456AD9023841
:10050000614440EA0840A0FB0294A1EB0E01A14225
:10051000C846A64656D353D05DB1B3EB080261EB93
:100520000E0101FA07F722FA06F3F1401F43C5E96D
:10053000007100263146BDE8F087C2F12003D840A3
:100540000CFA02FC21FA03F3914001434FEA1C47E5
:100550001FFA8CFEB3FBF7F007FB10360B0C43EAD7
:10056000064300FB0EF69E4204FA02F408D91CEB87
:10057000030300F1FF382FD29E422DD90238634485
:100580009B1B89B2B3FBF7F607FB163341EA034125
:1005900006FB0EF38B4208D91CEB010106F1FF3874
:1005A00016D28B4214D9023E6144C91A46EA00466B
:1005B00038E72E46284605E70646E3E61846F8E6FD
:1005C0004B45A9D2B9EB020864EB0C0E0138A3E746
:1005D0004646EAE7204694E74046D1E7D0467BE727
:1005E000023B614432E7304609E76444023842E79F
:1005F000704700BF02E000F000F8FEE772B637482F
:1006000080F30888364880F3098836483649086000
:1006100040F20000CCF200004EF63471CEF2000140
:100620000860BFF34F8FBFF36F8F40F20000C0F23E
:10063000F0004EF68851CEF200010860BFF34F8FF4
:10064000BFF36F8F4FF00000E1EE100A4EF63C71E1
:10065000CEF200010860062080F31488BFF36F8F8C
:1006600005F01AF805F01CF94FF055301F491B4AE8
:1006700091423CBF41F8040BFAE71D49184A9142E8
:100680003CBF41F8040BFAE71A491B4A1B4B9A423C
:100690003EBF51F8040B42F8040BF8E7002018495C
:1006A000184A91423CBF41F8040BFAE705F032F8D2
:1006B00005F078F9144C154DAC4203DA54F8041BDC
:1006C0008847F9E700F042F8114C124DAC4203DACA
:1006D00054F8041B8847F9E705F01AB80006002013
:1006E000002200200000000808ED00E000000020CB
:1006F00000060020E062000800220020A022002066
:10070000A0220020086F0020E0020008E402000898
:10071000E4020008E40200082DE9F04F2DED108AF4
:10072000C1F80CD0D0F80CD0BDEC108ABDE8F08F29
:10073000002383F311882846A047002004F0F0FB33
:10074000FEE704F053FB00DFFEE70000F8B501F020
:1007500053F904F025FF074604F094FF0546B8BBA3
:10076000204B9F4234D001339F4234D027F0FF0208
:100770001D4B9A4232D12E4642F21074F8B200F06C
:1007800071FF00F075FF08B10024264601F022FD3C
:1007900020B10024032000F07BF8264635B1134B2E
:1007A0009F4203D0002404F065FF2646002004F099
:1007B00001FF0EB100F082F801F0ECFA00F08CFFBE
:1007C00001F0CAF9204600F00BF900F077F8F9E7DC
:1007D0002E460024D5E704460126D2E7064641F21C
:1007E0008834CEE7010007B0000008B0263A09B00F
:1007F00008B501F07DF9A0F120035842584108BD29
:1008000007B541F21203022101A8ADF8043001F04E
:100810008DF903B05DF804FB38B5302383F31188FC
:10082000174803680BB104F039FC0023154A4FF454
:100830007A71134804F028FC002383F31188124CCA
:10084000236813B12368013B2360636813B16368B5
:10085000013B63600D4D2B7833B963687BB902208F
:1008600001F02EFA322363602B78032B07D16368E3
:100870002BB9022001F024FA4FF47A73636038BD7B
:10088000A022002019080008C0230020B822002060
:10089000084B187003280CD8DFE800F008050208A0
:1008A000022001F00BBA022001F006BA024B00222E
:1008B0005A607047B8220020C0230020F8B501F02C
:1008C00089FC30B13E4B03221A7000223D4B5A6026
:1008D000F8BD3D4B3D4A1C4619680131F8D0043340
:1008E0009342F9D162683A4B9A42F1D9394B9B68ED
:1008F00003F1006303F580239A42E9D204F08EFEEF
:1009000004F0A0FE002001F04DF90220FFF7C0FF27
:10091000314B00219A6C99641A6F19671A6FDA6C5F
:10092000D9645A6F59675A6F1A6D19659A6F99672A
:100930009B6F72B64FF0E023C3F8084DD4E9000472
:10094000BFF34F8FBFF36F8F244AC2F88410BFF3F9
:100950004F8F536923F480335361BFF34F8FD2F825
:10096000803043F6E076C3F3C905C3F34E335B0131
:1009700003EA060C29464CEA81770139C2F8747201
:10098000F9D2203B13F1200FF2D1BFF34F8FBFF309
:100990006F8FBFF34F8FBFF36F8F536923F4003313
:1009A00053610023C2F85032BFF34F8FBFF36F8FF4
:1009B000302383F31188854680F30888204787E732
:1009C000B8220020C02300200000040820000408F2
:1009D000FFFF0308002200200045025800ED00E060
:1009E0002DE9F04F93B0B74B2022FF2100900AA8C9
:1009F0009D6801F079F9B44A1378A3B90121B3488D
:100A000011700360302383F3118803680BB104F085
:100A100045FB0023AE4A4FF47A71AC4804F034FB36
:100A2000002383F31188009B13B1AA4B009A1A602C
:100A3000A94A1378032B03D000231370A54A5360EF
:100A40004FF0000A009CD3465646D146012001F0E3
:100A500035F924B19F4B1B68002B00F02C8200203D
:100A600001F046F80390039B002B01DA00F088FEAA
:100A7000039B002BEDDB012001F01EF9039B213BC2
:100A80001F2BE3D801A252F823F000BF0D0B000882
:100A9000350B0008C90B00084D0A00084D0A000874
:100AA0004D0A00085B0C00082B0E0008450D0008DD
:100AB000A70D0008CF0D0008F50D00084D0A00082D
:100AC000070E00084D0A0008790E0008AD0B00085B
:100AD0004D0A0008BD0E0008190B0008AD0B0008F8
:100AE0004D0A0008A70D00084D0A00084D0A00082D
:100AF0004D0A00084D0A00084D0A00084D0A00087A
:100B00004D0A00084D0A0008C90B00080220FFF733
:100B10006FFE002840F0F981009B022105A8BAF180
:100B2000000F08BF1C4641F21233ADF8143000F03C
:100B3000FDFF8BE74FF47A7000F0DAFF071EEBDB66
:100B40000220FFF755FE0028E6D0013F052F00F2F6
:100B5000DE81DFE807F0030A0D10133605230421B8
:100B600005A8059300F0E2FF17E004215548F9E7D6
:100B700004215A48F6E704215948F3E74FF01C08CE
:100B8000404608F1040801F00FF80421059005A87B
:100B900000F0CCFFB8F12C0FF2D101204FF000098A
:100BA00000FA07F747EA0B0B5FFA8BFB01F0E8F856
:100BB00026B10BF00B030B2B08BF0024FFF720FE20
:100BC00044E704214748CDE7002EA5D00BF00B03E6
:100BD0000B2BA1D10220FFF70BFE074600289BD06C
:100BE0000120002600F0DEFF0220FFF751FE1FFA71
:100BF00086F8404600F0E6FF0446B0B1039940464F
:100C00000136A1F140025142514100F0F3FF0028AA
:100C1000EDD1BA46044641F21213022105A83E4620
:100C2000ADF8143000F082FF10E725460120FFF7F1
:100C30002FFE244B9B68AB4207D9284600F0B4FF37
:100C4000013040F067810435F3E70025224BBA46B6
:100C50003E461D701F4B5D60A8E7002E3FF45CAF61
:100C60000BF00B030B2B7FF457AF0220FFF710FEA6
:100C7000322000F03DFFB0F10008FFF64DAF18F054
:100C800003077FF449AF0F4A08EB050392689342CC
:100C90003FF642AFB8F5807F3FF73EAF124BB84505
:100CA000019323DD4FF47A7000F022FF0390039A42
:100CB000002AFFF631AF039A0137019B03F8012B9D
:100CC000EDE700BF00220020BC230020A02200206E
:100CD00019080008C0230020B822002004220020A8
:100CE000082200200C220020BC220020C820FFF790
:100CF0007FFD074600283FF40FAF1F2D11D8C5F127
:100D000020020AAB25F0030084494245184428BF5D
:100D10004246019200F0D6FF019AFF217F4800F081
:100D2000E3FF4FEAA803C8F387027C4928460193F2
:100D300000F0E2FF064600283FF46DAF019B05EB93
:100D4000830533E70220FFF753FD00283FF4E4AEAC
:100D500000F062FF00283FF4DFAE0027B846704B7A
:100D60009B68BB4218D91F2F11D80A9B01330ED0A4
:100D700027F0030312AA134453F8203C059340467E
:100D8000042205A9043701F00FFA8046E7E7384648
:100D900000F00AFF0590F2E7CDF81480042105A8C1
:100DA00000F0C4FE02E70023642104A8049300F0CD
:100DB000B3FE00287FF4B0AE0220FFF719FD002833
:100DC0003FF4AAAE049800F01DFF0590E6E700236B
:100DD000642104A8049300F09FFE00287FF49CAED9
:100DE0000220FFF705FD00283FF496AE049800F0BE
:100DF0000BFFEAE70220FFF7FBFC00283FF48CAE74
:100E000000F01AFFE1E70220FFF7F2FC00283FF4B0
:100E100083AE05A9142000F015FF074604210490B5
:100E200004A800F083FE3946B9E7322000F060FEE6
:100E3000071EFFF671AEBB077FF46EAE384A07EBB4
:100E40000903926893423FF667AE0220FFF7D0FC99
:100E500000283FF461AE27F003074F44B9453FF443
:100E6000A5AE484609F1040900F09EFE0421059054
:100E700005A800F05BFEF1E74FF47A70FFF7B8FCCD
:100E800000283FF449AE00F0C7FE002844D00A9B7A
:100E900001330BD008220AA9002000F02DFF002802
:100EA0003AD02022FF210AA800F01EFFFFF7A8FC7D
:100EB0001C4804F03BF813B0BDE8F08F002E3FF45F
:100EC0002BAE0BF00B030B2B7FF426AE002364211B
:100ED00005A8059300F020FE074600287FF41CAE0D
:100EE0000220FFF785FC804600283FF415AEFFF78F
:100EF00087FC41F2883004F019F8059800F05EFF95
:100F000046463C4600F03CFFA0E506464EE64FF064
:100F1000000901E6BA467EE637467CE6BC220020A0
:100F200000220020A0860100094A49F269001368E6
:100F300099B21B0C00FB013344F250611360054B66
:100F4000186882B2000C01FB0200186080B2704782
:100F500014220020102200200021102210B5044687
:100F600000F0C2FE034B03CB206061601868A060F4
:100F700010BD00BF00E8F11F2DE9F041ADF54E7D39
:100F80000D46002140F275126CAC07460EA80D917B
:100F900000F0AAFE4FF4C4720021204600F0A4FE27
:100FA0000DF1340802F0C2FA4FF47A72264BB0FB0E
:100FB000F2F0186093E80700022384E807000DF5BB
:100FC000E9702382FFF7C8FF41F204331F4907A8E5
:100FD000238405F011F815230DF2E3220DF12C0CFA
:100FE00084F8323107AB1E46083203CE664542F81C
:100FF000080C42F8041C3346F5D1306841461060B5
:10100000204633791371012200F0F2FE002380B2F2
:10101000E97E0393AB7E029305F11903019301234B
:10102000009307A3D3E90023CDE90480384602F0FA
:101030003BFE0DF54E7DBDE8F08100BFAFF30080B3
:101040009E6AC421818A46EEC823002008600008F9
:101050002DE9F0412C4CDAB080460D46237A5BBB7B
:1010600027A9284600F0D2FF0746002842D19DF864
:101070009D60C82E3ED801464FF4A662204600F07F
:1010800033FE4FF4807332460DF19E01C4F8F831FF
:101090004FF4007304F109002644C4F80C334FF4F4
:1010A0004073C4F8203400F00DFE9DF89C30777238
:1010B00023720BB9EB7E237206AC8122002127A894
:1010C00000F012FE0122214627A800F0DBFF0023DA
:1010D00080B2E97E0393AB7E029305F1190301937D
:1010E0002823CDE904400093404605A3D3E900231B
:1010F00002F0DAFD5AB0BDE8F08100BFAFF3008026
:1011000026417272DF25D7B7905D0020F0B5254EDD
:101110004FF48A75F1B0002405FB006596F8D830CD
:10112000D822214685F8DC303AA885F8E84006AF99
:1011300000F0DAFD06F1090000F0CEFDD5F8E4304C
:10114000C2B206F109018DF8F0000DF1F100CDE910
:101150003A3400F0B7FD394601223AA800F0BEFF4C
:10116000082380B2317ACDE9047001270E48CDE919
:10117000023706F1D80301933023009307A3D3E984
:10118000002302F091FDA04206DD02F0CFF9C5F880
:10119000E000384671B0F0BD2046FBE778F6339F9B
:1011A00093CACD8D905D0020E03300202DE9F04FF3
:1011B000264F87B0DFF8A080254E384602F0A0FD0C
:1011C000034600283AD00024224DADF81440A14631
:1011D0000294A246CDE90344027B8DF8142003AAB1
:1011E0009968406803C21B6843F0004302932B6870
:1011F00004F5A664D3F810B002F09AF910EB0802D7
:10120000CDF800A0284605F5A65541F1000302A936
:10121000D8470028C8BF49F00109B4F5266FE6D1C8
:10122000B9F1000F05D0384602F06EFD86F800A037
:10123000C3E73378072B04D80133337007B0BDE818
:10124000F08F024802F060FDF8E700BFE0330020B5
:10125000C56200201034002040420F0070B50D46DA
:1012600014461E4602F07CFC50B9022E10D1012C0F
:101270000ED112A3D3E900230120C5E9002307E022
:10128000282C10D005D8012C09D0052C0FD0002017
:1012900070BD302CFBD10BA3D3E90023ECE70BA3EB
:1012A000D3E90023E8E70BA3D3E90023E4E70BA38A
:1012B000D3E90023E0E700BFAFF30080401DA12089
:1012C00026812A0B78F6339F93CACD8D9E6AC4215E
:1012D000818A46EE26417272DF25D7B7F017304A71
:1012E00039059E5638B505460E4C0021013500F0F3
:1012F00081FCA4F82C55B4F82C0500F063FC78B1FF
:10130000B4F82C0500F06EFC014648B9B4F82C0581
:1013100000F070FCB4F82C350133A4F82C35EAE762
:1013200038BD00BF905D0020F8B50D4C02260D4F72
:10133000A4F5805343F8307C237E3BB965692DB119
:10134000284600F0C5FF284604F00CFE2046A4F510
:10135000A65400F0BDFF012E00D1F8BD0126E7E73D
:1013600000590020C06000082DE9F04F8FB00546FD
:101370000C4600AF02F0F4FB002849D1237E022B7B
:101380001BD1E38A012B18D102F0D0F80646FFF7F3
:10139000CBFD03464FF4C87006F51676DFF8C08221
:1013A000B3FBF0F202FB103316FA83F3C8F80030F7
:1013B000E37E33B9A34B00221A703C37BD46BDE82B
:1013C000F08F07F12401204600F0DEFD0028F4D163
:1013D00007F11400FFF7C0FD97F8264007F114014C
:1013E00007F12700224604F0D5FD0028E2D10F2C9A
:1013F00008D8944B1C70D8F80030A3F51673C8F8C1
:101400000030DAE797F82410284602F0A1FBD4E771
:10141000E38A282B2BD010D8012B23D0052BCCD13D
:10142000BFF34F8F8849894BCA6802F4E0621343C7
:10143000CB60BFF34F8F00BFFDE7302BBDD1844E93
:10144000E17E327A9142B8D1607E3146002291F835
:10145000DC50854200F0A580013201F58A71042A32
:10146000F5D1AAE721462846FFF786FDA5E72146E4
:101470002846FFF7EDFDA0E7B2F8EC507B6005F1E0
:1014800003094FEA99094FEA8902D11DC908A8EB5F
:10149000C10300219D46EB46584600F025FC04F1AF
:1014A000EE012A465846314400F00CFC7B6813B923
:1014B000012000F077FB96F8D20000F083FB044691
:1014C00030B9307200F0A8FB204600F06BFBB1E0B1
:1014D000D6F8D4203AB996F8D200B6F82C25824234
:1014E00001D8FFF7FFFED6F8D4202A44944208D250
:1014F00096F8D200B6F82C250130824201D8FFF7C9
:10150000F1FE5FFA89F25946706800F0F5FB08B900
:10151000C54679E0726896F8D2002A447260D6F81F
:10152000D42005EB0209C6F8D49000F04BFB8145AE
:1015300009D396F8D220D6F8D4000132001B86F8E1
:10154000D220C6F8D400FF2D0FD80024347200F04A
:1015500063FB204600F026FB00F03CFE3D4B18816B
:1015600008B9FFF7ABF9C54627E7BB6896F8D9007D
:101570000AFB0362FB68D2F8E41082F8E83001F558
:101580008061C2F8E030C2F8E410FFF7BFFDFFF75A
:101590000DFE96F8D920013202F0030286F8D92018
:1015A000B6E74FF48A7A20460AFB02F505F1EA0114
:1015B000314400F0BFFDF86000287FF4FEAE012248
:1015C000354485F8E82001F0B1FFD5F8E020D6EDEC
:1015D000007A801A40F6B832B8EE677ADFED1E6AFC
:1015E000192838BF1920904228BF104607EE900AEC
:1015F000F8EEE77A67EEA67ADFED186AE7EE267A6C
:10160000FCEEE77AC6ED007A96F8D930BB60BA688E
:1016100073680AFB02F4321992F8E81059B1D2F853
:10162000E410E8468B423FF427AF002182F8E8102F
:10163000C2F8E010C5467368064A9B0A013313815D
:10164000BBE600BFD933002000ED00E00400FA053E
:10165000905D0020C8230020CDCCCC3D6666663F5F
:10166000DC330020014B1870704700BFD4230020EA
:1016700038B54FF04054144B22689A4221D1627D14
:101680000025124B12481A70C922237D09301149D6
:1016900000F8013C4FF48073C0F8DB50C0F8EF3124
:1016A0004FF40073C0F803334FF44073C0F817349D
:1016B00000F008FBE0222946204600F015FB01203F
:1016C00038BD0020FCE700BF9AAD44C5D4230020FC
:1016D000905D00201600003037B500F07BFD1F4CF8
:1016E0001F4D022301221F496B7123682881204668
:1016F0005B68984704F5805301221A49D3F8C03437
:1017000004F5A6505B689847002317494FF48052B0
:101710000193164B16480093164B02F0F1F9164B45
:10172000197811B1124802F013FA01F0FFFE0446D5
:10173000FFF7FAFB4FF4C873B0FBF3F202FB13039D
:1017400004F5167010FA83F00C4B186003F09AFF42
:1017500008B10F232B8103B030BD00BF103400202F
:10176000C823002040420F00D82300205D1200084B
:10177000E033002069130008D4230020DC3300206C
:101780002DE9F04F00242DED028B93B00DF12C08C4
:101790004FF0010ADFF814B2FFF708FD0A94ADF824
:1017A00034400B94C8F804409FED798B00267E4DA1
:1017B00037462B680DF11D0207A928468DF81CA09D
:1017C0008DF81D408DED008BD3F808900023C8479D
:1017D0009DF81C90B9F1000F1ED0102200210EA818
:1017E00000F082FA2B6808AA0AA95F6928460DF161
:1017F0001E03B8470FAB4F4698E8030083E8030089
:101800009DF834300EA958468DF844300A9B0E934B
:10181000DDE9082302F056FC06F5A66605F5A65597
:10182000B6F5266FC5D1002FC0D1604802F098F9F7
:1018300000283FD15E4E01F079FE3368984239D3DB
:1018400001F074FE0546FFF76FFB4FF4C8738DF887
:101850002870B0FBF3F202FB130305F5167010FAC3
:1018600083F03060534E377817B901238DF8283054
:10187000C7F110050EA8FFF76FFB0EABEDB20DF12F
:101880002900D919062D28BF06252A46013500F062
:1018900019FA0AABEDB24548039318230495029355
:1018A000454B0193012300933BA3D3E9002302F0AE
:1018B0009DF9347001F03AFE404A414D1368C31A55
:1018C000B3F57A7F2FD3106001F032FE02460B464B
:1018D000364802F023FA354802F042F918B32B7A61
:1018E0000EAF384E002B14BF03230223737101F097
:1018F0001DFE4FF47A7301223946B0FBF3F03060DD
:10190000304600F019FB182380B202932E4B01934E
:1019100040F25513CDE903700093244820A3D3E986
:10192000002302F063F92B7A93B101F0FFFD00264A
:1019300007464FF48A7895F8D900304400F0030048
:1019400008FB005393F8E82072B10136042EF2D15F
:10195000C82003F0EBFA2B7A002B7FF417AF13B0FB
:10196000BDEC028BBDE8F08FD3F8E02042B12B68CC
:10197000BA1AFA2B38BFFA230533B2EB430FE4D37C
:10198000FFF7C4FB0028E0D1E2E700BFAFF300801F
:101990000000000000000000401DA12026812A0B4D
:1019A000F1C6A7C1D068080F10340020E033002032
:1019B000DC330020D9330020D8330020C06200205F
:1019C000905D0020C8230020C462002010B5074CA1
:1019D000204601F0B1F804F5A65001F0ADF8044A34
:1019E00004490020BDE8104004F0B6BA10340020CD
:1019F0002063002029130008F8B50A25204C012295
:101A00004FF400712046192702F0EAFD204601221A
:101A10004FF4807102F0E4FD4FF4807665200138C8
:101A200025D00822A2F10801B646332905D84FF087
:101A3000000C66834FF000730DE0A1F13403668360
:101A4000B3FBF7FC07FB1C33002B0CBF4FF0010C62
:101A50004FF0000CEED1013143EA4C238A42A361DE
:101A6000A4F818E0E1D10832A02AD8D0DAE7013D85
:101A700042F2107003F05AFA15F0FF05BFD1F8BD1D
:101A8000000402582DE9F84F4FF47A7306460D46CC
:101A9000002402FB03F7DFF85080DFF8509098F93C
:101AA00000305FFA84FA5A1C01D0A34212D159F8CF
:101AB00024002A4631460368D3F820B03B46D84775
:101AC000854207D1074B012083F800A0BDE8F88FBD
:101AD0000124E4E7002CFBD04FF4FA7003F026FA5F
:101AE0000020F3E70C630020182200201C220020B5
:101AF000002307B5024601210DF107008DF80730DC
:101B0000FFF7C0FF20B19DF8070003B05DF804FBAC
:101B10004FF0FF30F9E700000A46042108B5FFF74F
:101B2000B1FF80F00100C0B2404208BD074B0A4639
:101B300030B41978064B53F82140014623682046FB
:101B4000DD69044BAC4630BC604700BF0C6300202D
:101B50001C220020A086010070B5104C0025104EFC
:101B600003F0A4FB20803068238883420CD8002532
:101B70002088013803F096FB23880544013BB5F526
:101B8000802F2380F4D370BD03F08CFB33680544B1
:101B90000133B5F5802F3360E5D3E8E70E6300200D
:101BA000C862002003F050BC00F1006000F5802006
:101BB0000068704700F10060920000F5802003F09B
:101BC000D1BB0000054B1A68054B1B889B1A83424A
:101BD00002D9104403F066BB00207047C8620020A1
:101BE0000E630020024B1B68184403F061BB00BF6A
:101BF000C8620020024B1B68184403F06BBB00BF97
:101C0000C86200200020704700F1FF5000F58F10DF
:101C1000D0F8000870470000064991F8243033B12D
:101C200000230822086A81F82430FFF7C3BF01208F
:101C3000704700BFCC620020014B1868704700BF9E
:101C40000010005C194B01380322084470B51D6870
:101C5000174BC5F30B042D0C1E88A6420BD15C68F4
:101C60000A46013C824213460FD214F9016F4EB16D
:101C700002F8016BF6E7013A03F10803ECD1814267
:101C80000B4602D22C2203F8012B0424094A1688A1
:101C9000AE4204D1984284BF967803F8016B013CB0
:101CA00002F10402F3D1581A70BD00BF0010005CAD
:101CB000242200204C60000870470000704700009C
:101CC00070470000002310B5934203D0CC5CC4548D
:101CD0000133F9E710BD000003460246D01A12F99D
:101CE000011B0029FAD1704702440346934202D0F7
:101CF00003F8011BFAE770472DE9F8431F4D14461E
:101D00000746884695F8242052BBDFF870909CB3B4
:101D100095F824302BB92022FF2148462F62FFF787
:101D2000E3FF95F824004146C0F1080205EB80006E
:101D3000A24228BF2246D6B29200FFF7C3FF95F811
:101D40002430A41B17441E449044E4B2F6B2082E7B
:101D500085F82460DBD1FFF75FFF0028D7D108E0CA
:101D60002B6A03EB82038342CFD0FFF755FF002895
:101D7000CBD10020BDE8F8830120FBE7CC62002036
:101D8000024B1A78024B1A70704700BF0C63002098
:101D90001822002010B5074C4FF4E13306492068A3
:101DA0000B6002F089FF60680349BDE8104002F053
:101DB00083BF00BF1C220020F4620020094B1822C0
:101DC000002110B504461846FFF78EFF064A074B60
:101DD00001461278046053F82200BDE8104002F07A
:101DE0006BBF00BFF46200200C6300201C220020A7
:101DF0002DE9F0470D46044600219046284640F262
:101E00007912FFF771FF234620220021284604F1B2
:101E1000220702F0F9F8231D022220212846C026BD
:101E200002F0F2F8631D03222221284602F0ECF8AA
:101E3000A31D03222521284602F0E6F804F1080339
:101E400010222821284602F0DFF804F110030822AE
:101E50003821284602F0D8F804F111030822402165
:101E6000284602F0D1F804F112030822482128463E
:101E700002F0CAF804F1140320225021284602F08F
:101E8000C3F804F1180340227021284602F0BCF880
:101E900004F120030822B021284602F0B5F804F12D
:101EA00021030822B821284602F0AEF83146083650
:101EB0003B4608222846013702F0A6F8B6F5A07F77
:101EC000F4D1002704F1330A04F132030822314629
:101ED000284602F099F894F832304FEAC7099F4239
:101EE00009F5A47615D3B8F1000F08D1314609F2EF
:101EF0004F1604F599730722284602F085F8274605
:101F00003B1B94F8322193420CD3F01DC008BDE86E
:101F1000F0870AEB0703082231462846013702F012
:101F200073F8D8E707F233133146082228460836FB
:101F3000013702F069F8E3E713B5044608460021CB
:101F40002022234601900160C0F8031002F05CF8E3
:101F5000231D01980222202102F056F8631D0198EA
:101F60000322222102F050F8A31D0198032225210B
:101F700002F04AF8019804F108031022282102F027
:101F800043F8072002B010BD0023F7B50E46047FCA
:101F9000072200911946054601F0FAFE731C012242
:101FA000072100932846002301F0F2FEC4B9B31CB8
:101FB000052208212846009323460D2401F0E8FE5F
:101FC0003746BB1BB278934211D307342B7FA88AC4
:101FD000E408BBB9844294BF0020012003B0F0BDE7
:101FE000AB8A0824DB00083BDB08B370E8E7FB1C86
:101FF000214608222846009300230834013701F0C7
:10200000C7FEDEE7201A18BF0120E7E70023F7B577
:102010000E46047F082200911946054601F0B8FEDD
:10202000731CC4B908220093234610241146284685
:1020300001F0AEFE01235F1C7278013B934211D385
:1020400007342B7FA88AE408BBB9844294BF0020E0
:10205000012003B0F0BDAB8A0824DB00083BDB089D
:102060007370E7E7F31921460822284600930023FE
:1020700001F08EFE08343B46DDE7201A18BF012030
:10208000E7E70000F8B50E46054614460021812218
:102090003046FFF729FE2B4608220021304601F08A
:1020A000B3FF7CB90F246B1C07220821304601F0D6
:1020B000ABFF01235F1C6A78013B934204D3E01D10
:1020C000C008F8BD0824F4E7EB1921460822304681
:1020D00001F09AFF08343B46ECE70000F8B50E46E5
:1020E000054614460021CE223046FFF7FDFD2B4663
:1020F00028220021304601F087FF7CB9302405F109
:10210000080308222821304601F07EFF2F467B1B62
:102110002A7A934204D3E01DC008F8BD2824F5E7CD
:1021200007F109032146082230460834013701F03F
:102130006BFFECE7F7B5047F0E46009101231022F8
:102140000021054601F024FEC4B9B31C0922102168
:10215000284600932346192401F01AFE3746728858
:10216000BB1B9A4211D807342B7FA88AE408BBB95D
:10217000844294BF0020012003B0F0BDAB8A10243C
:10218000DB00103BDB087380E8E73B1D214608229B
:102190002846009300230834013701F0F9FDDEE7FB
:1021A000201A18BF0120E7E730B50A44084D9142D4
:1021B0000DD011F8013B5840082340F30004013BC7
:1021C0002C4013F0FF0384EA5000F6D1EFE730BD56
:1021D0002083B8EDF7B5384A6B46106851686A46F7
:1021E00003C308233549364803F0E4FE04460028BB
:1021F00033D10A25334A6B46106851686A4603C3D7
:10220000082331492E4803F0D5FE0446002849D062
:102210000369B3F5E01F45D8B0F8661040F21342E9
:1022200091423FD1294A024402F15C018B4239D3E9
:102230005C3B234900209E1AFFF7B6FF04F16401BE
:10224000074632460020FFF7AFFFA3689F4229D11F
:10225000E368984208BF002524E00369B3F5E01F56
:1022600027D8418B40F21342914220D1174A0244B1
:1022700002F110018B4218D3103B114900209D1A26
:10228000FFF792FF04F1180106462A460020FFF7E7
:102290008BFFA3689E4202D1E368984201D00D25CE
:1022A000A8E70025284603B0F0BD1025A2E70C25BD
:1022B000A0E70B259EE700BF5C600008DCFF1B0069
:1022C000000004086560000890FF1B000800FCF790
:1022D00010B5037C044613B9006803F053FE204692
:1022E00010BD00000023BFF35B8FC360BFF35B8FA3
:1022F000BFF35B8F8360BFF35B8F7047BFF35B8F70
:102300000068BFF35B8F704770B505460C30FFF770
:10231000F5FF044605F108063046FFF7EFFFA0423F
:1023200006D96D683046FFF7E9FF2544281A70BDCD
:102330003046FFF7E3FF201AF9E7000070B50546C5
:102340004068A0B105F10C0605F10800FFF7D6FFC3
:1023500004463046FFF7D2FF844204F1FF34304692
:1023600094BF6D680025FFF7C9FF2C44201A70BD8B
:1023700038B50C460546FFF7C7FFA04210D305F15C
:102380000800FFF7BBFF04446868BFF35B8FB4FB32
:10239000F0F100FB11440120AC60BFF35B8F38BD4E
:1023A0000020FCE72DE9F041144607460D46FFF7F3
:1023B000C5FF844228BF0446D4B1B84658F80C6B18
:1023C0004046FFF79BFF3044286040467E68FFF799
:1023D00095FF331A9C4203D801206C60BDE8F08160
:1023E000A41B6B603B682044AB60E8600220F5E70B
:1023F0002046F3E738B50C460546FFF79FFFA0429D
:1024000010D305F10C00FFF779FF04446868BFF3AF
:102410005B8FB4FBF0F100FB11440120EC60BFF3D3
:102420005B8F38BD0020FCE72DE9FF4188466946F7
:1024300007466C46FFF7B6FF002506B204EBC6065A
:10244000B4420AD0626808EB050120680834FFF73F
:1024500039FC54F8043C1D44F2E729463846FFF79E
:10246000C9FF284604B0BDE8F0810000F8B5054674
:102470000C300F46FFF742FF05F1080604463046D0
:10248000FFF73CFFA042304688BF6C68FFF736FF7D
:10249000201A386020B12C683046FFF72FFF204407
:1024A000F8BD000073B5144606460D46FFF72CFF35
:1024B0008442019028BF0446DCB101A93046FFF7F1
:1024C000D5FF019B33B93268C5E90233C5E9002461
:1024D00001200CE09C42286038BF0194019884429E
:1024E0006860F5D93368241A0220AB60EC6002B052
:1024F00070BD2046FBE700002DE9FF410F4669460D
:102500006C46FFF7CFFF00B2002604EBC005AC42DB
:1025100009D0D4F80480B81954F8081B4246464440
:10252000FFF7D0FBF3E7304604B0BDE8F0810000D0
:1025300038B50546FFF7E0FF044601462846FFF799
:1025400017FF204638BD0000302383F3118862B6A0
:1025500070470000002383F3118862B670470000C3
:10256000012070477047000010B4134602681468D9
:102570000022A4465DF8044B6047000000F580503F
:1025800090F859047047000000F5805090F852040C
:102590007047000000F5805090F958047047000023
:1025A0004E20704700F5805208B5FFF7CDFFD2F8F6
:1025B0009C34D2F898041844D2F894341844D2F8D1
:1025C0007C341844D2F88C341844D2F88834184437
:1025D000FFF7C0FF08BD00002DE9F04F0C4600F5E5
:1025E000805185B01F4691F8523405469046BDF89B
:1025F00038909BB1D1F878340133C1F8783423682E
:102600009A0006D4237B082B0BD9627B0AB10F2BCF
:1026100007D9D1F87C340133C1F87C344FF0FF3056
:102620000FE0FFF791FFEB6AD3F8C42012F4001A11
:102630000AD0D1F8803400200133C1F88034FFF78C
:1026400089FF05B0BDE8F08F22684FF0480BD3F842
:10265000C460002A6B6AC6F30446B4BF42F08042ED
:1026600092041BFB063BCBF8002023685B004FEA7B
:10267000066344BF42F00052CBF80020227B43EABD
:1026800002437201CBF80430607B18B343F440136B
:10269000CBF80430D1F8B0340133C1F8B034AB1802
:1026A00003F58353197B41F020011973207B0392BA
:1026B00000F098FF0330039A80105FFA8AF30AF162
:1026C000010A83420DDA04EB83010BEB83034968B3
:1026D0009960F2E7AB1803F58353197B60F345115A
:1026E000E3E70121EB6A04F10C00B140C3F8D0101C
:1026F000AB18214603F58253C3E9048705EB461363
:1027000003F58253183351F804CB814243F804CBCC
:10271000F9D109882A442846198041F26803D65025
:1027200002F5805209F0030392F86C1043F0100395
:1027300021F01F010B43214682F86C304246FFF71F
:1027400009FF3B46CDF8009000F012FF012078E72A
:102750002DE9F04700F58056044696F85254002DB6
:1027600040F00181037C032B40F092802B462846E9
:102770002F465FFA83FC944510DA01EBCC0E51F83A
:102780003CC0BCF1000F04DBDEF804C0BCF1000F5C
:1027900002DB01370133ECE70130FBE7FFF7D4FE42
:1027A000E36AF0B9D3F8800040F00200C3F880007B
:1027B0004E23E06A002F6ED1D0F8803043F0010341
:1027C000C0F88030694B6A4A1B6803F1805303F5F7
:1027D0002C539B009342A36240F2AF80654800F007
:1027E0009FFE4D2842D8DFF884814FEA004EDFF883
:1027F0008891D8F800C04EEA8C0EC3F884E00CF142
:10280000805303F52C539B00636100EB0C03D4F859
:102810002CC0C8F80030C0F14E03DCF8800040F056
:102820003000CCF880004FF0000CD4F81480E6465D
:102830005FFA8CF08242BCDD01EBC00A51F8300037
:10284000002810DBDAF804A0BAF1000F0BDA09EA6D
:1028500000400AF07F0A40EA0A0040F0084048F8C9
:102860002E000EF1010E0CF1010CE1E79A6922F045
:1028700001029A6100F05AFE0646E36A9B69D90795
:1028800004D500F053FE831BFA2BF6D9FFF762FE46
:102890002846BDE8F087B7EB530F3DD2DFF8CCE018
:1028A0004FEA074CDEF800304CEA830CC0F888C0D1
:1028B00003F1805003EB4703002700F52C50CEF8BE
:1028C0000030BC468000A061E06AD0F8803043F060
:1028D0000C03C0F88030D4F818E0FBB29A427FF7BE
:1028E00071AF51F8330001EBC3080028D8F8043069
:1028F00001DB002B0EDB20F0604023F0604340F052
:10290000005043F000434EF83C000EEBCC000CF1BD
:10291000010C43600137E0E7836923F00103836121
:1029200000F004FE0646E36A9B69DA07AED500F0C4
:10293000FDFD831BFA2BF6D9A8E7E26A936923F021
:102940000103936100F0F2FD0746E36A9B69DB0730
:1029500005D500F0EBFDC31BFA2BF6D996E7012550
:1029600086F8525492E7002592E700BF1C630020CE
:10297000FCB50040706000080000FF0713B500F5CB
:1029800080540191606CFFF7D9FC1F280AD92022DE
:102990000199606CFFF748FDA0F1200358425841AF
:1029A00002B010BD0020FBE700F5805008B5FFF72E
:1029B000CBFD406CFFF796FCBDE80840FFF7CABDB1
:1029C0000022026082814260826070470022002300
:1029D00010B5C0E90023002304460C3020F8043C65
:1029E000FFF7EEFF204610BD2DE9F047074688B0FF
:1029F0009A46884607F5805468469146FFF7A4FD3D
:102A0000FFF7E4FF606CFFF77FFC1F282DD9202221
:102A10006946606CFFF78CFD202826D194F852346B
:102A20001BB303AD444605AB2E46083403CE9E428D
:102A300044F8080C44F8041C3546F5D1306841468A
:102A400020603846B388A380DDE90023C9E900236C
:102A5000BDF808304A46AAF80030FFF77BFD534620
:102A600008B0BDE8F04700F071BD0020FFF772FD2F
:102A700008B0BDE8F08700002DE9F84F00230646B6
:102A800000F58154054688461034C0E90133274BD0
:102A900046F8303B374638462037FFF797FFA742C6
:102AA000F9D105F580544FF4805305F5A3594FF043
:102AB000000A26630026676405F5835709F11009AB
:102AC0004FF0000B1037E663C4E90D36012384F89C
:102AD000403084F84830A7F11800203747E910ABA0
:102AE000FFF76EFF47F8286C4F45F4D1B8F1010F9E
:102AF00084F85884A4F85A64A4F85C64A4F85E646A
:102B000084F86064A4F86264A4F86464A4F8666459
:102B100084F8686402D9064800F002FD054B284697
:102B200053F82830EB62BDE8F88F00BFC0600008A2
:102B300094600008B0600008044B10B51978044692
:102B40004A1C1A70FFF798FF204610BD1963002039
:102B50002DE9F04700295FD0304F3148B7FBF1F540
:102B600081428CBF0A201120431EB5FBF0FC00FB04
:102B70001C50DCB220B1022B1846F5D8002037E0FB
:102B80000CF1FF35B5F5806F32D2C4EBC4094FF4B8
:102B90007A7009F103034FEAE308C3F3C70308F1AE
:102BA000010AA4EB030E08FB00085FFA8EF65AFA3E
:102BB0008EFEB8FBFEFEBEF5617F1BDC1FFA8EF4B5
:102BC000581C56FA80F00CFB00FCB7FBFCFC61457E
:102BD000D4D1013BDBB20F2BD0D8711E0020C9B27B
:102BE000072905D810710120148055805371917107
:102BF000BDE8F08709F1FF334FEAE30EC3F3C703E3
:102C00000EF10108E41A0EFB0000E6B258FA84F453
:102C1000B0FBF4F4A4B2D3E70846E9E700B4C40477
:102C20003F420F0038B540F27772C36A154CC3F8C3
:102C3000BC200722C36AC3F8C8202268C16A930077
:102C400043F4C023C1F8A03002F1805302F16C01BB
:102C5000C56A03F52C53EA3289009B00226041F0DB
:102C6000E061094AC361C5F8C01003F5D87103F5E6
:102C70006A7341629342836202D9044800F050FCB7
:102C800038BD00BF1C630020FCB500407060000828
:102C90002DE9F04F00F58055994689B0044695F826
:102CA00058348A469046022B04D90027384609B08A
:102CB000BDE8F08F9B4A52F8231009B942F823006F
:102CC0009949C4F80CA00B7884F81090C3B9FFF7A9
:102CD0003BFC964BD3F8EC2042F48072C3F8EC2016
:102CE000D3F8942042F48072C3F89420D3F894204F
:102CF00022F48072C3F8942001230B70FFF72AFCA2
:102D000095F851346BB9FFF71FFC894A95F8583490
:102D1000D35CEBB1012B24D0012385F85134FFF7AC
:102D200019FCFFF711FCE26A936923F01003936129
:102D300000F0FCFB0746E36A9E6916F0080617D010
:102D400000F0F4FBC31BFA2BF5D9FFF703FCACE74B
:102D50000321132001F0FAFD0321152001F0F6FDF7
:102D6000DAE70321142001F0F1FD03211620F5E735
:102D70009A6942F001029A6100F0D8FB0746E36AC3
:102D80009A69D00705D400F0D1FBC31BFA2BF6D902
:102D9000DBE79A69002704F5825B42F002020BF13F
:102DA000100B9A61E36A5F65FFF7D4FB686CFFF76D
:102DB00099FA202200216846FEF796FF02A8FFF745
:102DC000FFFD6A460BEB06030DF1180E06979446BD
:102DD0000833BCE80300F44543F8080C43F8041C2E
:102DE0006246F4D1DCF8000020361860B6F5806F3A
:102DF0009CF804201A71DCD1002304F5A25251463C
:102E000020461A3285F8503485F85334FFF7A0FE77
:102E1000074690B9E26A936923F00103936100F0D9
:102E200085FB0546E36A9B69D9077FF53EAF00F055
:102E30007DFB431BFA2BF5D937E795F85F6495F8CE
:102E40005E243602C5F86CA4E36A46EA426695F849
:102E500060241643B5F85C2446EA0246DE61B8F108
:102E6000000F29D004F5A352414620460232FFF755
:102E70006FFE90B9E26A936923F00103936100F059
:102E800055FB0546E36A9B69DA077FF50EAF00F054
:102E90004DFB431BFA2BF5D907E795F8683495F8F5
:102EA00067141B01C5F87084E26A43EA0123B5F890
:102EB000641443EA0143D360E36A00262046C3F862
:102EC000BC60FFF7AFFE85F859646FF04042E36ADB
:102ED0001A65184AE36A5A654FF00222E36A9A6556
:102EE0004FF0FF32E36AC3F8E0200322E36A914522
:102EF000DA653FF4DBAEE26A936923F00103936184
:102F000000F014FB0646E36A9B69DB0705D500F079
:102F10000DFB831BFA2BF6D9C7E6012385F8523443
:102F2000C4E600BF1063002018630020004402586C
:102F3000A8600008550200022DE9F04F054689B04F
:102F400090469946002741F2680A00F58056EB6AE0
:102F5000D3F8D830FB40D8074ED505EB47124FEADF
:102F6000471B52441379190746D4D6F884340133E9
:102F7000C6F8843405F5A553C3E9008913799A0688
:102F800005EB0B0248BFD6F8B434524444BF0133BA
:102F9000C6F8B434137943F008031371DB0723D563
:102FA00096F8533403B305F582546846FFF70EFDD7
:102FB00003AB18345C4404F1080C2068083454F85E
:102FC000041C1A46644503C21346F6D120686946BC
:102FD00010602846A2889A800123ADF808302B683B
:102FE000CDE90089DB6B9847D6F8543423B1D6F885
:102FF000A8340133C6F8A8340137202FA7D109B06F
:10300000BDE8F08F2DE9F04F0F468DB0044600F07B
:103010008FFA82468946002F5BD1E36AD3F8A0205D
:1030200012F4FE0F03D100200DB0BDE8F08FD3F8ED
:10303000A420920141BF04F58051D1F898240132B7
:10304000C1F89824D3F8A4205606ECD0D3F8A450A5
:10305000E669C5F305254823E8464FF0000B03FB5E
:1030600005664046FFF7ACFC326851004ABF22F0CB
:103070006043C2F38A4343F00043920048BF43F0E9
:1030800080430093736813F400131BBF012304F5FE
:1030900080528DF80D308DF80D301EBFD2F8B83447
:1030A0000133C2F8B834F38803F00F038DF80C3005
:1030B0009DF80C0000F096FA5FFA8BF3984225D940
:1030C000F2180CA90BF1010B127A0B4403F82C2C0B
:1030D000EEE7012FA7D1E36AD3F8B02012F4FE0F78
:1030E000A1D0D3F8B420950141BF04F58051D1F8A7
:1030F00098240132C1F89824D3F8B420500692D015
:10310000D3F8B450266AC5F30525A4E7EFB9E36AFE
:10311000C3F8A85004A807ADFFF758FC98E80F00C3
:1031200007C52B800023204604A9ADF8183023687A
:1031300004F58054DB6BCDE904A9984758B1D4F865
:1031400090340133C4F890346EE7012FE2D1E36A82
:10315000C3F8B850DEE7D4F8943401200133C4F842
:10316000943461E7F8B505460F4600F58054012612
:1031700039462846FFF746FF10B184F85364F7E755
:10318000D4F8543423B1D4F8A8340133C4F8A834A3
:10319000F8BD0000C36AF0B51A6C12F47F0F2BD093
:1031A0001B6C00F5805441F268054FF0010CC4F827
:1031B000AC340023471900EB43125E012A44117915
:1031C00011F0020F15D0490713D4B959C66A0CFA89
:1031D00001F1D6F8CCE011EA0E0F0AD0C6F8D410EF
:1031E000117941F004011171D4F88C240132C4F832
:1031F0008C240133202BDED1F0BD00002B4B70B5A9
:103200001E561B5C012B30D8294D2A4A55F8233015
:1032100052F8264013B349B3236D9A0510D54FF4E5
:103220000073236500F084F950EA01020B4602D0D6
:10323000013861F10003024655F82600FFF77CFED5
:10324000236D9B012CD54FF0007255F82630226576
:1032500003F58053012283F8592421E001232365DB
:10326000102323654FF48053236570BD236DDA0767
:1032700002D4236D5B0706D50523002155F82600EF
:103280002365FFF76FFF236DD80602D4236D59061F
:1032900006D55023012155F826002365FFF762FF6C
:1032A00055F82600BDE87040FFF774BFAC60000819
:1032B00010630020B060000808B5FFF745F9FFF77C
:1032C00069FFBDE80840FFF745B90000C36AD3F8BD
:1032D000C00010F07C5005D0D3F8C40080F400107A
:1032E000C0F340507047000000F5805008B5FFF76C
:1032F0002BF9406CFFF708F8FFF72CF943090CBFD6
:103300000120002008BD000000F5805393F85924E7
:1033100062B1C16A8A6922F001028A61D3F89C24F1
:103320000132C3F89C24002283F85924704700001E
:103330002DE9F74300F5825198460025FFF704F97F
:10334000103141F2680E4FF0010900F5805C00EB8E
:103350004514744423795E071CD4DB061AD58E69A4
:10336000C36A09FA06F6D3F8CC703E4212D04F6811
:1033700001970F689742019F77EB08070AD2C3F8BD
:10338000D460237943F004032371DCF888340133DB
:10339000CCF8883401352031202DD8D103B0BDE8D8
:1033A000F043FFF7D7B80000F8B51E4600230F46DC
:1033B000054613701446FFF797FF80F00100387040
:1033C0001EB12846FFF782FF2070F8BD2DE9F04FAF
:1033D00085B099460D468046164691F800B0DDE965
:1033E0000EA302931378019300F0A2F82B78044601
:1033F0000F4613B93378002B42D022463B46404655
:10340000FFF796FFFFF758FFFFF77EFF4B46324668
:103410002946FFF7C9FF2B7833B1BBF1000F03D06A
:10342000012005B0BDE8F08F337813B1019B002B6C
:10343000F6D108F5805303935445029B77EB0303C1
:103440001ED2039BD3F85404D0B10368AAEB040145
:10345000DB6889B298474B46324629464046FFF71B
:10346000A3FF2B7813B1BBF1000FD9D1337813B17F
:10347000019B002BD4D100F05BF804460F46DBE73C
:103480000020CEE7002108B50846FFF7B7FEBDE8EB
:10349000084001F06DB8000008B501210020FFF7D9
:1034A000ADFEBDE8084001F063B8000008B500219A
:1034B0000120FFF7A3FEBDE8084001F059B8000065
:1034C000012108B50846FFF799FEBDE8084001F064
:1034D0004FB8000000B59BB0EFF309816822684641
:1034E000FEF7F0FBEFF30583014B9B6BFEE700BF9C
:1034F00000ED00E008B5FFF7EDFF000000B59BB060
:10350000EFF3098168226846FEF7DCFBEFF30583E1
:10351000014B5B6BFEE700BF00ED00E0FEE7000043
:103520000FB408B5029801F097FCFEE701F0D8BF90
:1035300001F0B0BF13B56C46031D84E8060094E8A3
:10354000030083E80500012002B010BD73B5856853
:10355000019155B11B885B0707D4D0E900369B6BFE
:103560009847019AC1B23046A847012002B070BD09
:10357000F0B5866889B005460C465EB1BDF83830B6
:103580005B070AD4D0E900379B6B98472246C1B24B
:103590003846B047012009B0F0BD0022002301F1F8
:1035A0000806CDE9002300230A46ADF8083003AB36
:1035B0001068083252F8041C1C46B24203C4234669
:1035C000F6D1106820609288A280FFF7B1FF042333
:1035D000ADF808302B68CDE90001DB6B6946284661
:1035E0009847D7E7082817D909280CD00A280CD003
:1035F0000B280CD00C280CD00D280CD00E2814BF92
:103600004020302070470C20704710207047142055
:103610007047182070472020704700002DE9F041C6
:10362000456A15B94162BDE8F0814B68AC4623F0AC
:103630006047C3F38A464FEAD37EC3F3807816EA25
:10364000230638BF3E462B465A68BEEBD27F22F097
:1036500060440AD0002A18DAA40CB44217D19D4263
:103660000FD10D60DEE71346EEE7A74207D102F067
:103670008044C2F3807242450BD054B1EFE708D2C8
:10368000EDE7CCF800100B60CDE7B44201D0B442B6
:10369000E5D81A689C46002AE5D11960C3E7000006
:1036A0002DE9F047089D01F0070400EBD1004FF42D
:1036B0007F494FEAD508224405F00705944201D11D
:1036C000BDE8F08704F0070705F0070A111B08EBB7
:1036D000D50E57453E4613F80EC038BF5646C6F1C4
:1036E00008068E4228BF0E46E108415C344435444A
:1036F000B94029FA06F721FA0AF1FFB28CEA010172
:1037000047FA0AF739408CEA010C03F80EC0D5E7F6
:1037100080EA0120082341F2210201B2013B40006E
:10372000002980B2B8BF504013F0FF03F5D17047B5
:1037300038B50C468D18A54200D138BD14F8011BD0
:10374000FFF7E6FFF7E7000042684AB11368818996
:103750004360438901339BB29942438138BF8381DF
:103760001046704770B588B0044620220D46684662
:103770000021FEF7B9FA20460495FFF7E5FF02465F
:1037800060B16B46054608AE1C46083503CCB44212
:1037900045F8080C45F8041C2346F5D1104608B03E
:1037A00070BD0000082817D909280CD00A280CD0B1
:1037B0000B280CD00C280CD00D280CD00E2814BFD0
:1037C0004020302070470C20704710207047142094
:1037D000704718207047202070470000082817D92C
:1037E0000C280CD910280CD914280CD918280CD95D
:1037F00020280CD930288CBF0F200E2070470920BC
:1038000070470A2070470B2070470C2070470D202E
:10381000704700002DE9F843078C0446072F1ED996
:1038200000254FF6FF73D0E90298C5F12006A5F1F7
:10383000200029FA05F1083508FA06F628FA00F002
:10384000314301431846C9B2FFF762FF402D0346DA
:10385000EBD13A46E169BDE8F843FFF769BF4FF69F
:10386000FF70BDE8F883000010B54B6823B9CA8A21
:1038700063F30902CA8210BD04691A681C600361FF
:10388000C38A013BC3824A60EFE700002DE9F84F8D
:103890001D46CB8A0F468146C3F30901924605298E
:1038A0000B4630D00020AAB207F11A049EB21FFACC
:1038B00080F8042E0FD8904503F1010306D30A4483
:1038C000FB8A62F309030120FB821AE01AF8006008
:1038D0000130E654EAE79045F1D2A1F1050B1C2333
:1038E0007C68BBFBF3F203FB12BB1FFA8BF6002CC8
:1038F00045D14846FFF728FF044638B978606FF095
:103900000200BDE8F88F4FF00008E6E700260660E9
:103910007860ADB24FF0000B454510D90AEB0803B3
:10392000221D13F8011B08F101089155B1B21FFACD
:1039300088F81B292BD0454506F10106F1D8FB8AF2
:10394000C3F30902154465F30903BCE701321C46C1
:1039500092B22368002BF9D16B1F0B441C21B3FBDF
:10396000F1F301339BB29A42D3D2BBF1000FD0D115
:103970004846FFF7E9FE20B9C4F800B0BFE70122CE
:10398000E7E7C0F800B05E4620600446C1E7454561
:10399000D5D94846FFF7D8FE08B92060AFE7C0F890
:1039A00000B0002620600446B6E700002DE9F04F85
:1039B0001C46074688462DED028B83B05B69019259
:1039C000002B00F09A80238C2BB1E269002A00F0D2
:1039D0009480072B35D807F10C00FFF7B5FE05469C
:1039E00038B96FF00205284603B0BDEC028BBDE884
:1039F000F08F14220021FEF777F9228CE16905F19E
:103A00000800FEF75FF9208C48F00041013080B2D9
:103A1000FFF7E4FEFFF7C6FE013880B220840130D4
:103A2000287438466369228C1B782A4403F01F03EC
:103A300063F03F03137269602946FFF7EFFD01252C
:103A4000D1E74FF0000900F10C034FF0800A4E4619
:103A50004D4608EE103A18EE100AFFF775FE834641
:103A60000028BED014220021FEF73EF9002E3AD1E4
:103A7000019B0222ABF808300BF1080E1FFA82FC02
:103A8000218C0CF10100BCF1060F80B201D88E42EE
:103A90002BD3FFF7A3FE8E4208BF4FF0400AFFF77B
:103AA00081FE62690138013512781BFA80F101301C
:103AB00002F01F022DB242EA491289F001094AEAD6
:103AC000020A48F0004281F808A059468BF810001D
:103AD0003846CBF804204FF0000AFFF79FFD238CF7
:103AE000B342B8D17FE70022C6E7E169895D0136BC
:103AF0000EF80210B6B20132C0E76FF0010572E7AE
:103B0000F8B515460E463022002104461F46FEF742
:103B1000EBF8069BB5F5001FA760636004F1100089
:103B2000079B34BF6A094FF6FF72E661A362002368
:103B300097B29A4206D800230360A782E3822383C8
:103B4000E360F8BD0660013330462036F1E700003F
:103B500003781BB94BB2002BC8BF0170704700003F
:103B600000787047F8B50C46C969074611B9238C2F
:103B7000002B37D1257E1F2D34D8387828BB228CD6
:103B8000072A2CD8268A36F003032BD14FF6FF7074
:103B9000FFF7CEFD20F0010031024FF6FF72400426
:103BA00041EA0561400C41EA402523462946384652
:103BB000FFF7FCFE002807DD626913780133DBB2F2
:103BC0001F2B88BF00231370F8BD218A2D0645EAFC
:103BD000012505432046FFF71DFE0246E5E76FF08D
:103BE0000300F1E76FF00100EEE7000070B58AB066
:103BF000044616460021282268461D46FEF774F842
:103C0000BDF8383069462046ADF810300F9B05935B
:103C10009DF840308DF81830119B0793BDF848305F
:103C2000CDE90265ADF82030FFF79CFF0AB070BD0A
:103C30002DE9F041D36905460C4616460BB9138CA5
:103C40005BBB377E1F2F28D895F80080B8F1000F96
:103C500026D03046FFF7DEFD3378210202462846A3
:103C600041EAC331338A41EA080141EA076141EA86
:103C70000341334641F08001FFF798FE00280ADD3A
:103C80003378012B07D1726913780133DBB21F2B14
:103C900088BF00231370BDE8F0816FF00100FAE7E0
:103CA0006FF00300F7E70000F0B58BB004460D4657
:103CB00017460021282268461E46FEF715F89DF893
:103CC0004C30294620465A1E534253416A468DF8CD
:103CD00000309DF84030ADF81030119B05939DF8F1
:103CE00048308DF81830149B0793BDF85430CDE957
:103CF0000276ADF82030FFF79BFF0BB0F0BD00005F
:103D0000406A00B104307047436A1A68426202692F
:103D10001A600361C38A013BC38270472DE9F041F9
:103D2000D0F8208014461D46184E4146002709B998
:103D3000BDE8F081D1E90223A21A65EB03039642A4
:103D400077EB03031ED2036A8B420DD1FFF78CFD84
:103D5000036A1B68036203690B60C38A0161013B4C
:103D6000016AC3828846E2E7FFF77EFD0B68C8F868
:103D7000003003690B60C38A0161013BC382D8F83C
:103D80000010D4E788460968D1E700BF80841E0090
:103D90002DE9F04F8BB00D4614469B46DDF8509050
:103DA0008046002800F01881B9F1000F00F014815E
:103DB000531E3F2B00F21081012A03D1BBF1000FEB
:103DC00040F00A810023CDE90833B8F81430B5EB90
:103DD000C30F4FEAC30703D300200BB0BDE8F08F39
:103DE0002B199F42D8F80C3036BF7F1B2746FFB2F5
:103DF0001BB9D8F81030002B7AD0272D4DD8C5F13B
:103E0000280600232946B742009308ABD8F80800DB
:103E10002CBFF6B23E46A7EB060A354432465FFA9F
:103E20008AFAFFF73DFCB8F81430282103F100535B
:103E3000053BDB000493D8F80C300393039B13B1CC
:103E4000BAF1000F2CD1D8F8100040B1BAF1000F30
:103E500005D008AB5246691A0096FFF721FC38B22C
:103E6000002FB9D066070AD00AAB624203EBD40137
:103E700002F0070211F8083C134101F8083C082C35
:103E80003DD9102C40F2B580202C40F2B780BBF118
:103E9000000F00F09C80082335E0BA460026C2E7F8
:103EA000049BE02B28BFE02306930B44AB42059311
:103EB00015D95A1B0398691A0096924508AB00F170
:103EC000040034BF5246D2B20792FFF7E9FB079ACB
:103ED0001644AAEB020A1544F6B25FFA8AFA049B6A
:103EE000069A05999B1A0493039B1B680393A5E705
:103EF00000933A4608AB2946D8F80800ADE7BBF175
:103F0000000F13D00123B4EBC30F6BD0082C12D8D1
:103F10009DF82030621E23FA02F2D50706D54FF035
:103F2000FF3202FA04F423438DF820309DF820304C
:103F300089F8003051E7102C12D8BDF82030621EED
:103F400023FA02F2D10706D54FF0FF3202FA04F449
:103F50002343ADF82030BDF82030A9F800303CE70D
:103F6000202C0FD80899631E21FA03F3DA0705D530
:103F70004FF0FF3202FA04F40C430894089BC9F88E
:103F800000302AE7402C2AD0611EC4F12102A4F19E
:103F90002103DDE9086526FA01F105FA02F225FAA6
:103FA00003F311431943CB0711D50122A4F12003D8
:103FB000C4F1200102FA03F322FA01F1A2400B43FB
:103FC000524263EB430332432B43CDE90823DDE93F
:103FD0000823C9E9002300E76FF00100FDE66FF058
:103FE0000800FAE6082CA1D9102CB4D9202CEED860
:103FF000C4E7BBF1000FAED0022384E7BBF1000F92
:10400000BCD004237FE70000012A30B5144638BF36
:10401000012485B00025402C28BF4024012ACDE989
:10402000025518D81B788DF8083063070AD004AB06
:10403000624203EBD40502F0070215F8083C9340F6
:1040400005F8083C034600912246002102A8FFF72C
:1040500027FB05B030BD082AE4D9102A03D81B88F5
:10406000ADF80830E1E7202A95BF1B68D3E90023AB
:104070000293CDE90223D8E710B5CB681BB98B605A
:104080000B618B8210BD04691A681C600361C38ACE
:10409000013BC382CA60F0E703064CBFC0F3C030E7
:1040A0000220704708B50246FFF7F6FF022806D146
:1040B0005306C2F30F2001D100F0030008BDC2F384
:1040C0000740FBE72DE9F04F93B004460D46CDE9DC
:1040D00003230A681046FFF7DFFF0228824614BF59
:1040E000C2F306260026002A80F2F38112F0C049AE
:1040F00040F0EF81097B002900F0EB81022803D01A
:104100002378B34240F0E881C2F3046310462944A7
:10411000069302F07F030593FFF7C4FF059B00227F
:1041200083464FEA8348002348EA0A4848EA46683B
:10413000CE78CDE90823F30948EA0008029368D055
:10414000059B024608A92046009353466768B84776
:10415000002800F0C481276A4FB9414604F10C00E1
:10416000FFF700FB074690B96FF0020055E03B698E
:1041700098450DD03F68002FF9D1414604F10C005D
:10418000FFF7F0FA07460028EED0236A3B6027626B
:1041900097F817C006F01F08CCF3840CACEB0800AE
:1041A000A8EB0C031FFA80FE0028B8BF0EF1200018
:1041B0001FFA83FEB8BF00B2002B0793B8BF0EF101
:1041C0002003D7E90221BCBF1BB2079352EA0103C7
:1041D00038D0039B4FF0000CDFF820E39A1A049BC1
:1041E00063EB010196457CEB01032BD36B7B97F8C6
:1041F0001AE0734519D1029B002B78D0012821DCED
:104200007868F8B9DFF8F0C2944570EB010316D373
:1042100037E0276A27B96FF00C0013B0BDE8F08FC4
:104220003B699845B4D03F68F4E7B34890427CEBD3
:10423000010301D30020F0E7029B002BFAD0079B7B
:104240000F2B17DCFA7DB3003946204602F003023B
:1042500003F07C031343FB75FFF706FB6B7BBB7618
:10426000029B3BB9FB7DC3F38402013262F38603F8
:10427000FB75D0E76A7BBB7E9A42DBD1029B002BA9
:1042800035D0B309022B32D0039B142200210DA894
:10429000BB60049BFB60FDF727FD039B0AA920463A
:1042A0000A93049BADF83EB00B932B1D8DF840A0F4
:1042B0000C932B7B8DF84180013BDBB2ADF83C3099
:1042C000069B8DF84230059B8DF8433094F82C30D6
:1042D00083F001038DF84430A3689847FB7DC3F356
:1042E0008403013303F01F039B02FB82A2E7FB7DE3
:1042F000C6F34012B2EBD31F40F0F480C3F3840343
:10430000434540F0F280029AB6092B7B002A4DD03B
:10431000F2075DD4032B40F2EB80039BAE1D3946C0
:1043200004F10C00BB603246049BFB602B7B033B1B
:10433000DBB2FFF7ABFA00280CDA39462046FFF76C
:1043400093FAFB7DC3F38403013303F01F039B0245
:10435000FB8209E7AB88DDE908843B834FF6FF73F6
:10436000C9F12000A9F1200228FA09F109F1080990
:1043700004FA00F024FA02F2014318461143C9B2CC
:10438000FFF7C6F9B9F1400F0346E9D1B8823146CB
:104390002A7B033AD2B2FFF7CBF9FB7DB882DA432E
:1043A000C2F3C01262F3C713FB7543E786B92E1D33
:1043B000013B394604F10C00DBB23246FFF766FAE6
:1043C0000028BADB2A7B3146B88A013AD2B2E2E74A
:1043D000F98A013BC1F30901DAB204295BD8281D2F
:1043E000002307F11B069A4208D910F801CB0133CC
:1043F00006F801C00131DBB20529F4D103999342DB
:104400000A9138BF043304992CBF002355FA83F373
:104410000B9107F11B010C9179680E930D91291DE9
:10442000FB8AADF83EB0C3F309038DF840A08DF8C8
:1044300041801A44069B8DF84230059BADF83C2024
:104440008DF8433094F82C3083F001038DF844301C
:104450000023B88A7B602A7B013AFFF769F93B8B1E
:10446000B882834203D1A3680AA920469847204610
:104470000AA9FFF701FEFB7DBA8AC3F38403013367
:1044800003F01F039B02FB823B8B9A420CBF002070
:104490006FF01000C1E67B68002BAFD0052001E073
:1044A0001C3033461E68002EFAD1091A2E1D081D35
:1044B000184401EB090C5FFA89F3BCF11B0F9DD87E
:1044C0009A429BD916F8013B09F1010900F8013B1A
:1044D000EFE76FF00900A0E66FF00A009DE66FF0CD
:1044E0000B009AE66FF00D0097E66FF00E0094E671
:1044F0006FF00F0091E600BF40420F0080841E0065
:10450000EFF30983054968334A6B22F001024A63DD
:1045100083F30988002383F31188704700EF00E0DC
:10452000302080F3118862B60D4B0E4AD96821F411
:10453000E0610904090C0A430B49DA60D3F8FC2056
:1045400042F08072C3F8FC20084AC2F8B01F11681C
:1045500041F0010111602022DA7783F822007047D0
:1045600000ED00E00003FA0555CEACC5001000E0F8
:10457000302310B583F311880E4B5B6813F400638E
:1045800014D0F1EE103AEFF309844FF08073683CD9
:10459000E361094BDB6B236684F3098800F01AFCA6
:1045A00010B1064BA36110BD054BFBE783F31188E7
:1045B000F9E700BF00ED00E000EF00E0430700086E
:1045C000460700080023054A19460133102BC2E9AB
:1045D000001102F10802F8D1704700BF24630020E7
:1045E0002DE9F74F02F0030AC2F3C313C2F38009A7
:1045F000C2F3C108C2F3411E574600224FF00F0B11
:104600000193CB0733D502F00703019C0125560027
:104610009B00BAF1020F05FA02F504FA03FC4468A4
:104620000BFA03F324EA05046FEA030344EA0904DE
:1046300044604FF00304856804FA06F625EA06058F
:104640006FEA060445EA08058560C56825EA06059F
:1046500045EA0E05C5601BD1072A13D8056A2B4011
:1046600043EA0C03036203681C403C4304604908AE
:1046700022D04FEA490901324FEA88084FEA8E0EEC
:10468000BF00BEE7456A2B4043EA0C034362EAE7FA
:104690000568072A04EA050444EA0704046005D80B
:1046A000046A234043EA0C030362E0E7446A2340C0
:1046B00043EA0C034362DAE703B0BDE8F08F000081
:1046C000026843681143016003B118477047000056
:1046D000024A136843F0C0031360704700100140A2
:1046E000024A136843F0C00313607047007C004027
:1046F00037B51A4C1A4D204600F0D2FA04F11400D6
:10470000009400234FF40072164900F08FF94FF423
:104710000072154904F138000094144B00F008FAB7
:10472000134BC4E91735134C204600F0B9FA04F1D5
:10473000140000234FF400720F49009400F076F942
:104740000E4B4FF400720E4904F13800009400F053
:10475000EFF90C4BC4E9173503B030BDA46300205A
:1047600000E1F5057C6400207C680020D14600084B
:1047700000100140106400207C660020E146000823
:104780007C6A0020007C0040037C30B5284C002966
:1047900018BF0C46012B0CD1264B984236D1264B24
:1047A0001A6D42F010021A659A6F42F010029A6771
:1047B0009B6F2268036EC16D03EB52038466B3FBEB
:1047C000F2F36268150442BF23F0070503F0070304
:1047D00043EA4503CB60A36843F040034B60E368C2
:1047E00043F001038B6042F4967343F001030B60C6
:1047F0004FF0FF330B62510505D512F0102213D094
:10480000B2F1805F12D080F8643030BD0B4B98421B
:10481000CFD1094B9A6C42F000429A641A6F42F071
:1048200000421A671B6FC4E77F23ECE73F23EAE7E8
:1048300000610008A46300200045025810640020B5
:104840002DE9F047C66D05463768F46921073462E3
:104850001AD014F0080118BF4FF48071E20748BF66
:1048600041F02001A3074FF0300348BF41F0400161
:10487000600748BF41F0800183F31188281DFFF7CE
:104880001FFF002383F31188E2050AD5302383F349
:1048900011884FF48061281DFFF712FF002383F376
:1048A00011884FF030094FF0000A14F0200838D179
:1048B0003B0616D54FF0300905F1380A200610D511
:1048C00089F31188504600F067F9002836DA08218C
:1048D000281DFFF7F5FE27F080033360002383F3E4
:1048E0001188790614D5620612D5302383F3118816
:1048F000D5E913239A4208D12B6C33B127F0400736
:104900001021281DFFF7DCFE3760002383F3118898
:10491000E30618D5AA6E1369ABB15069BDE8F0473C
:10492000184789F31188736A284695F8641019406E
:1049300000F0D0F98AF31188F469B6E7B06288F321
:104940001188F469BAE7BDE8F0870000090100F1B9
:104950006043012203F56143C9B283F8001300F0FC
:104960001F039A4043099B0003F1604303F5614331
:10497000C3F880211A607047F8B51546826804466E
:104980000B46AA4200D28568A1692669761AB5420B
:104990000BD218462A46FDF795F9A3692B44A3616B
:1049A0002846A3685B1BA360F8BD0CD9AF1B184653
:1049B0003246FDF787F93A46E1683044FDF782F95F
:1049C000E3683B44EBE718462A46FDF77BF9E368CA
:1049D000E5E7000083689342F7B50446154600D228
:1049E0008568D4E90460361AB5420BD22A46FDF731
:1049F00069F963692B4463612846A3685B1BA36064
:104A000003B0F0BD0DD93246AF1B0191FDF75AF945
:104A100001993A46E0683144FDF754F9E3683B44B4
:104A2000E9E72A46FDF74EF9E368E4E710B50A44E2
:104A30000024C361029B8460C16002610362C0E91B
:104A40000000C0E9051110BD08B5D0E90532934258
:104A500001D1826882B98268013282605A1C426147
:104A600019700021D0E904329A4224BFC36843611F
:104A700000F078FA002008BD4FF0FF30FBE700009F
:104A800070B5302304460E4683F31188A568A5B19E
:104A9000A368A269013BA360531CA3611578226936
:104AA000934224BFE368A361E3690BB120469847B2
:104AB000002383F31188284607E03146204600F0A2
:104AC00041FA0028E2DA85F3118870BD2DE9F74F2D
:104AD00004460E4617469846D0F81C904FF0300A10
:104AE0008AF311884FF0000B154665B12A4631460E
:104AF0002046FFF741FF034660B94146204600F0DB
:104B000021FA0028F1D0002383F31188781B03B029
:104B1000BDE8F08FB9F1000F03D001902046C847DF
:104B2000019B8BF31188ED1A1E448AF31188DCE790
:104B3000C160C361009B82600362C0E9051111443A
:104B4000C0E9000001617047F8B504460D461646FD
:104B5000302383F31188A768A7B1A368013BA36042
:104B600063695A1C62611D70D4E904329A4224BF01
:104B7000E3686361E3690BB120469847002080F346
:104B8000118807E03146204600F0DCF90028E2DA1F
:104B900087F31188F8BD0000D0E9052310B59A42CB
:104BA00001D182687AB982680021013282605A1C80
:104BB00082611C7803699A4224BFC368836100F054
:104BC000D1F9204610BD4FF0FF30FBE72DE9F74F3C
:104BD00004460E4617469846D0F81C904FF0300A0F
:104BE0008AF311884FF0000B154665B12A4631460D
:104BF0002046FFF7EFFE034660B94146204600F02D
:104C0000A1F90028F1D0002383F31188781B03B0A9
:104C1000BDE8F08FB9F1000F03D001902046C847DE
:104C2000019B8BF31188ED1A1E448AF31188DCE78F
:104C3000026843681143016003B1184770470000E0
:104C40001430FFF743BF00004FF0FF331430FFF77D
:104C50003DBF00003830FFF7B9BF00004FF0FF3311
:104C60003830FFF7B3BF00001430FFF709BF000072
:104C70004FF0FF311430FFF703BF00003830FFF76B
:104C800063BF00004FF0FF323830FFF75DBF000018
:104C9000012914BF6FF0130000207047FFF728BDF3
:104CA000044B036000234360C0E902330123037413
:104CB000704700BF1861000810B53023044683F325
:104CC0001188FFF761FD02230020237480F311880F
:104CD00010BD000038B5C36904460D461BB9042158
:104CE0000844FFF7A5FF294604F11400FFF7ACFEC6
:104CF000002806DA201D4FF40061BDE83840FFF7B8
:104D000097BF38BD00238268037503691B689968E3
:104D10009142FBD25A68036042601060586070474D
:104D200000238268037503691B6899689142FBD868
:104D30005A680360426010605860704708B50846C2
:104D4000302383F311880B7D032B05D0042B0DD06A
:104D50002BB983F3118808BD8B6900221A604FF0CC
:104D6000FF338361FFF7CEFF0023F2E7D1E9003282
:104D700013605A60F3E70000FFF7C4BF054BD96822
:104D800008751868026853601A600122D8600275BD
:104D9000FBF7C2BC806C00200C4B30B5DD684B1CAF
:104DA00087B004460FD02B46094A684600F06CF9DC
:104DB0002046FFF7E3FF009B13B1684600F06EF951
:104DC000A86907B030BDFFF7D9FFF9E7806C002074
:104DD0003D4D0008044B1A68DB6890689B68984258
:104DE00094BF002001207047806C0020084B10B554
:104DF0001C68D868226853601A600122DC60227542
:104E0000FFF78EFF01462046BDE81040FBF784BC4B
:104E1000806C0020044B1A68DB6892689B689A4299
:104E200001D9FFF7E3BF7047806C002038B5074C0D
:104E300001230025064907482370656000F0D8FC6F
:104E40000223237085F3118838BD00BFE86E00206F
:104E500044610008806C002008B572B6044B1865E8
:104E600000F006FB00F0D8FB024B03221A70FEE7AD
:104E7000806C0020E86E002000F046B9EFF311804E
:104E800020B9EFF30583302282F3118870470000C8
:104E900010B530B9EFF30584C4F3080414B180F3FE
:104EA000118810BDFFF7B6FF84F31188F9E7000001
:104EB0008B600223086108468B8270478368A3F1E8
:104EC000840243F8142C026943F8442C426943F8E5
:104ED000402C094A43F8242CC268A3F1200043F86F
:104EE000182C022203F80C2C002203F80B2C034A86
:104EF00043F8102C704700BF31070008806C002079
:104F000008B5FFF7DBFFBDE80840FFF735BF00003D
:104F1000024BDB6898610F20FFF730BF806C0020E8
:104F2000302383F31188FFF7F3BF000008B5014673
:104F3000302383F311880820FFF72EFF002383F32B
:104F4000118808BD064BDB6839B1426818605A60A9
:104F5000136043600420FFF71FBF4FF0FF3070471E
:104F6000806C00200368984206D01A680260506086
:104F700018469961FFF700BF70470000036810B53D
:104F80009C68A2420CD85C688A600B604C6021600F
:104F9000596099688A1A9A604FF0FF33836010BD98
:104FA000121B1B68ECE700000A2938BF0A2170B504
:104FB00004460D460A26601900F012FC00F0FAFBC8
:104FC000041BA54203D8751C04462E46F3E70A2E9F
:104FD00004D90120BDE8704000F04ABC70BD00005B
:104FE000F8B5144B0D460A2A4FF00A07D96103F1B0
:104FF0001001826038BF0A224160196914460160BD
:1050000048601861A81800F0DBFB00F0D3FB431BDD
:105010000646A34206D37C1C28192746354600F0D5
:10502000DFFBF2E70A2F04D90120BDE8F84000F0C9
:105030001FBCF8BD806C0020F8B506460D4600F098
:10504000B9FB0F4A134653F8107F9F4206D12A46F8
:1050500001463046BDE8F840FFF7C2BFD169BB68E2
:10506000441A2C1928BF2C46A34202D92946FFF71F
:105070009BFF224631460348BDE8F840FFF77EBF5C
:10508000806C0020906C0020C0E90323002310B442
:105090005DF8044B4361FFF7CFBF000010B5194C1A
:1050A000236998420DD08168D0E9003213605A60BC
:1050B0009A680A449A60002303604FF0FF33A361AB
:1050C00010BD0268234643F8102F5360002202608F
:1050D00022699A4203D1BDE8104000F07BBB93687F
:1050E00081680B44936000F065FB2269E169926876
:1050F000441AA242E4D91144BDE81040091AFFF74E
:1051000053BF00BF806C00202DE9F047DFF8BC8062
:1051100008F110072C4ED8F8105000F04BFBD8F8CF
:105120001C40AA68031B9A423ED814444FF0000961
:10513000D5E90032C8F81C4013605A60C5F80090E9
:10514000D8F81030B34201D100F044FB89F3118844
:10515000D5E9033128469847302383F311886B69DA
:10516000002BD8D000F026FB6A69A0EB0409824628
:105170004A450DD2022000F07BFB0022D8F8103007
:10518000B34208D151462846BDE8F047FFF728BF93
:10519000121A2244F2E712EB09092946384638BFB1
:1051A0004A46FFF7EBFEB5E7D8F81030B34208D017
:1051B0001444C8F81C00211AA960BDE8F047FFF7A5
:1051C000F3BEBDE8F08700BF906C0020806C00202B
:1051D00000207047FEE70000704700004FF0FF30EE
:1051E00070470000BFF34F8F044B1A695107FCD181
:1051F000D3F810215207F8D1704700BF00200052A9
:1052000008B50D4B1B78ABB9FFF7ECFF0B4BDA6819
:10521000D10704D50A4A5A6002F188325A60D3F89D
:105220000C21D20706D5064AC3F8042102F18832C0
:10523000C3F8042108BD00BFF06E0020002000521A
:105240002301674508B5114B1B78F3B9104B1A6958
:10525000510703D5DA6842F04002DA60D3F8102132
:10526000520705D5D3F80C2142F04002C3F80C21B7
:10527000FFF7B8FF064BDA6842F00102DA60D3F8B4
:105280000C2142F00102C3F80C2108BDF06E002091
:10529000002000520F289ABF00F5806040040020D3
:1052A000704700004FF40030704700001020704736
:1052B0000F2808B50BD8FFF7EDFF00F500330268A3
:1052C000013204D104308342F9D1012008BD00200D
:1052D000FCE700000F2838B505463FD8FFF782FFEE
:1052E0001F4CFFF78DFF4FF0FF3307286361C4F8B1
:1052F00014311DD82361FFF775FF030243F0240327
:10530000E360E36843F08003E36023695A07FCD459
:105310002846FFF767FFFFF7BDFF4FF4003100F0AD
:1053200057F92846FFF78EFFBDE83840FFF7C0BFAA
:10533000C4F81031FFF756FFA0F108031B0243F039
:105340002403C4F80C31D4F80C3143F08003C4F8C2
:105350000C31D4F810315B07FBD4D9E7002038BDFD
:10536000002000522DE9F84F05460C46104645EA4C
:105370000203DE0602D00020BDE8F88F20F01F00F7
:10538000DFF8BCB0DFF8BCA0FFF73AFF04EB000881
:10539000444503D10120FFF755FFEDE720222946C0
:1053A000204600F0F7FD10B920352034F0E72B46F9
:1053B00005F120021F68791CDDD104339A42F9D12E
:1053C00005F178431B481C4EB3F5801F1B4B38BFBB
:1053D000184603F1F80332BFD946D1461E46FFF7FF
:1053E00001FF0760A5EB040C336804F11C0143F0D6
:1053F00002033360231FD9F8007017F00507FAD1B4
:1054000053F8042F8B424CF80320F4D1BFF34F8F95
:10541000FFF7E8FE4FF0FF332022214603602846C5
:10542000336823F00203336000F0B4FD0028BBD0E2
:105430003846B0E7142100520C20005214200052CC
:10544000102000521021005210B5084C237828B1CA
:105450001BB9FFF7D5FE0123237010BD002BFCD034
:105460002070BDE81040FFF7EDBE00BFF06E0020D9
:1054700038B5054D00240334696855F80C0B00F06D
:10548000B9F8122CF7D138BD50610008084600F079
:1054900079BD000070B5104E82B0FFF7EFFC0546F5
:1054A00000F088F9326803469042336037BF0B4AF8
:1054B0000A495168146836BF0131D1E90041516091
:1054C0000419284641F100010191FFF7E1FC204653
:1054D000019902B070BD00BFF46E0020F86E00208C
:1054E00070B5124E82B0FFF7C9FC054600F062F9B4
:1054F000326803469042336037BF0D4A0C49516809
:10550000146836BF0131D1E90041516004192846C1
:1055100041F100010191FFF7BBFC4FF47A720023C7
:1055200020460199FAF7E4FE02B070BDF46E002047
:10553000F86E00200244074BD2B210B5904200D161
:1055400010BD441C00B253F8200041F8040BE0B237
:10555000F4E700BF504000580E4B30B51C6F2404D8
:1055600005D41C6F1C671C6F44F400441C670A4C74
:1055700002442368D2B243F480732360074B904205
:1055800000D130BD441C51F8045B00B243F82050F8
:10559000E0B2F4E700440258004802585040005876
:1055A00007B5012201A90020FFF7C4FF019803B04D
:1055B0005DF804FB13B50446FFF7F2FFA04205D0E7
:1055C000012201A900200194FFF7C6FF02B010BD1F
:1055D0000144BFF34F8F064B884204D3BFF34F8F74
:1055E000BFF36F8F7047C3F85C022030F4E700BF51
:1055F00000ED00E00144BFF34F8F064B884204D317
:10560000BFF34F8FBFF36F8F7047C3F87002203026
:10561000F4E700BF00ED00E070470000074B45F2E3
:1056200055521A6002225A6040F6FF729A604CF698
:10563000CC421A600122024B1A7070470048005891
:10564000046F0020034B1B781BB1034B4AF6AA22C0
:105650001A607047046F002000480058034B1A6816
:105660001AB9034AD2F8D0241A607047006F00209C
:1056700000400258024B4FF48032C3F8D0247047E8
:105680000040025808B5FFF7E9FF024B1868C0F365
:10569000806008BD006F002070B5BFF34F8FBFF36F
:1056A0006F8F1A4A0021C2F85012BFF34F8FBFF319
:1056B0006F8F536943F400335361BFF34F8FBFF3D0
:1056C0006F8FC2F88410BFF34F8FD2F8803043F64B
:1056D000E074C3F3C900C3F34E335B0103EA04066D
:1056E000014646EA81750139C2F86052F9D2203B81
:1056F00013F1200FF2D1BFF34F8F536943F480337E
:105700005361BFF34F8FBFF36F8F70BD00ED00E0AB
:10571000FEE70000214B2248224A70B5904237D361
:10572000214BC11EDA1C121A22F003028B4238BF31
:1057300000220021FCF7D8FA1C4A0023C2F884306A
:10574000BFF34F8FD2F8803043F6E074C3F3C90043
:10575000C3F34E335B0103EA0406014646EA817552
:105760000139C2F86C52F9D2203B13F1200FF2D16B
:10577000BFF34F8FBFF36F8FBFF34F8FBFF36F8FA9
:105780000023C2F85032BFF34F8FBFF36F8F70BD4D
:1057900053F8041B40F8041BC0E700BF80630008F7
:1057A000086F0020086F0020086F002000ED00E067
:1057B00000F01AB9014B586A704700BF000C004056
:1057C000034B002258631A610222DA60704700BF5F
:1057D000000C0040014B0022DA607047000C0040D2
:1057E000014B5863704700BF000C0040FEE700000B
:1057F00070B51B4B0025044686B058600E46856286
:105800000163FEF78DFE04F11003A560E562C4E9B3
:1058100004334FF0FF33C4E90044C4E90635FFF711
:10582000C9FF2B46024604F134012046C4E908238F
:1058300080230C4A2565FFF73BFB01230A4AE06001
:1058400000920375684672680192B268CDE902233E
:10585000064BCDE90435FFF753FB06B070BD00BF22
:10586000E86E0020986100089D610008ED5700086F
:10587000024AD36A1843D062704700BF806C002090
:105880004B6843608B688360CB68C3600B6943617E
:105890004B6903628B6943620B68036070470000C9
:1058A00008B53A4B40F2FF713948D3F888200A43D3
:1058B000C3F88820D3F8882022F4FF6222F0070280
:1058C000C3F88820D3F88830324B1A6C0A431A6424
:1058D0009A6E0A439A66304A9B6E1146FFF7D0FFD4
:1058E00000F5806002F11C01FFF7CAFF00F580603F
:1058F00002F13801FFF7C4FF00F5806002F15401A6
:10590000FFF7BEFF00F5806002F17001FFF7B8FFFE
:1059100000F5806002F18C01FFF7B2FF00F58060B6
:1059200002F1A801FFF7ACFF00F5806002F1C401AD
:10593000FFF7A6FF00F5806002F1E001FFF7A0FF8E
:1059400000F5806002F1FC01FFF79AFF02F58C710F
:1059500000F58060FFF794FF00F004F90F4BD3F8D7
:10596000902242F00102C3F89022D3F8942242F030
:105970000102C3F894220522C3F898204FF0605228
:10598000C3F89C20064AC3F8A02008BD0044025872
:105990000000025800450258A461000800ED00E034
:1059A0001F00080308B500F0C9FAFFF73FFA0B4BD8
:1059B000DA6B42F04002DA635A6E22F040025A6615
:1059C0005B6E074B1A6842F008021A601A6842F0D0
:1059D00004021A60BDE80840FFF740BE00450258C7
:1059E00000180248704700000E4B9A6C42F0080203
:1059F0009A641A6F42F008021A670B4A1B6FD36B46
:105A000043F00803D363C722084B9A624FF0FF327A
:105A1000DA6200229A615A63DA605A6001225A619E
:105A20001A607047004502580010005C000C0040EE
:105A3000094A08B51169D3680B40D9B29B076FEAD0
:105A40000101116107D5302383F31188FFF714FAA0
:105A5000002383F3118808BD000C0040044BDA6B6F
:105A60000243DA635A6E104358665B6E704700BF9C
:105A7000004502583A4B4FF0FF31D3F8802062F0D6
:105A80000042C3F88020D3F8802002F00042C3F81F
:105A90008020D3F88020D3F88420C3F88410D3F872
:105AA00084200022C3F88420D3F88400D86F40F00B
:105AB000FF4040F4FF0040F4DF4040F07F00D86733
:105AC000D86F20F0FF4020F4FF0020F4DF4020F0EA
:105AD0007F00D867D86FD3F888006FEA40506FEA2C
:105AE0005050C3F88800D3F88800C0F30A00C3F808
:105AF0008800D3F88800D3F89000C3F89010D3F84A
:105B00009000C3F89020D3F89000D3F89400C3F825
:105B10009410D3F89400C3F89420D3F89400D3F8E9
:105B20009800C3F89810D3F89800C3F89820D3F8D9
:105B30009800D3F88C00C3F88C10D3F88C00C3F80D
:105B40008C20D3F88C00D3F89C00C3F89C10D3F8B9
:105B50009C10C3F89C20D3F89C3000F0BFB900BF64
:105B60000044025808B50122504BC3F80821504B9D
:105B70005A6D42F002025A65DA6F42F00202DA67A9
:105B80000422DB6F4B4BDA605A689104FCD54A4A19
:105B90001A6001229A60494ADA6000221A614FF4C1
:105BA00040429A61434B9A699204FCD51A6842F4C8
:105BB00080721A60424B1A6F12F4407F04D04FF487
:105BC00080321A6700221A671A6842F001021A60CE
:105BD0003B4B1A685007FCD500221A611A6912F073
:105BE0003802FBD1012119604FF0804159605A679A
:105BF000344ADA62344A1A611A6842F480321A600E
:105C00002F4B1A689103FCD51A6842F480521A602F
:105C10001A689204FCD52D4A2D499A6200225A63D3
:105C2000196301F57C01DA6301F5E77199635A6440
:105C3000284A1A64284ADA621A6842F0A8521A609E
:105C40001F4B1A6802F02852B2F1285FF9D148229E
:105C50009A614FF48862DA6140221A621F4ADA645C
:105C60001F4A1A651F4A5A651F4A9A6532231F4AFE
:105C70001360136803F00F03022BFAD1104A136963
:105C800043F003031361136903F03803182BFAD1AF
:105C90004FF00050FFF7E2FE4FF08040FFF7DEFECE
:105CA0004FF00040BDE80840FFF7D8BE008000512B
:105CB000004502580048025800C000F004000001EE
:105CC000004402580000FF01008890083220600064
:105CD00063020901470E0508DD0BBF01200000200B
:105CE000000001100910E000000101100020005226
:105CF0004FF0B04208B5D2F8883003F00103C2F883
:105D0000883023B1044A13680BB150689847BDE846
:105D10000840FEF72DBC00BF246300204FF0B042C6
:105D200008B5D2F8883003F00203C2F8883023B1F6
:105D3000044A93680BB1D0689847BDE80840FEF765
:105D400017BC00BF246300204FF0B04208B5D2F862
:105D5000883003F00403C2F8883023B1044A136981
:105D60000BB150699847BDE80840FEF701BC00BF81
:105D7000246300204FF0B04208B5D2F8883003F019
:105D80000803C2F8883023B1044A93690BB1D06983
:105D90009847BDE80840FEF7EBBB00BF2463002036
:105DA0004FF0B04208B5D2F8883003F01003C2F8C3
:105DB000883023B1044A136A0BB1506A9847BDE892
:105DC0000840FEF7D5BB00BF246300204FF0B0436E
:105DD00010B5D3F8884004F47872C3F88820A3067D
:105DE00004D5124A936A0BB1D06A9847600604D56D
:105DF0000E4A136B0BB1506B9847210604D50B4A22
:105E0000936B0BB1D06B9847E20504D5074A136C2E
:105E10000BB1506C9847A30504D5044A936C0BB1A1
:105E2000D06C9847BDE81040FEF7A2BB2463002069
:105E30004FF0B04310B5D3F8884004F47C42C3F867
:105E40008820620504D5164A136D0BB1506D984732
:105E5000230504D5124A936D0BB1D06D9847E00429
:105E600004D50F4A136E0BB1506E9847A10404D5A8
:105E70000B4A936E0BB1D06E9847620404D5084A62
:105E8000136F0BB1506F9847230404D5044A936FE6
:105E90000BB1D06F9847BDE81040FEF769BB00BF5B
:105EA0002463002008B50348FEF7CAFCBDE808409B
:105EB000FEF75EBBA463002008B50348FEF7C0FCF4
:105EC000BDE80840FEF754BB1064002008B5FFF79A
:105ED000AFFDBDE80840FEF74BBB0000062108B54A
:105EE0000846FEF733FD06210720FEF72FFD0621A9
:105EF0000820FEF72BFD06210920FEF727FD0621CD
:105F00000A20FEF723FD06211720FEF71FFD0621BC
:105F10002820FEF71BFD09217A20FEF717FD072137
:105F20003220FEF713FD0C212520FEF70FFD0C217A
:105F30005320BDE80840FEF709BD000008B5FFF793
:105F400099FDFEF73FFBFEF7A9FEFFF74BFDBDE80D
:105F50000840FFF72DBC00000B460146184600F034
:105F600003B8000000F00EB810B5054C13462CB174
:105F70000A4601460220AFF3008010BD2046FCE730
:105F800000000000024B01461868FFF77FBA00BF0F
:105F90003C22002010B501390244904201D100207A
:105FA00005E0037811F8014FA34201D0181B10BD82
:105FB0000130F2E72DE9F041A3B1C91A1778014485
:105FC000044603F1FF3C8C42204601D9002009E041
:105FD0000578BD4204F10104F5D10CEB0405D61897
:105FE000A54201D1BDE8F08115F8018D16F801ED4B
:105FF000F045F5D0E7E70000034611F8012B03F860
:10600000012B002AF9D17047636F6D2E63756265AD
:1060100070696C6F742E6865726534666300000089
:1060200053544D333248373F3F3F0053544D333282
:10603000483733782F3732780053544D333248374E
:1060400034332F3735332F373530000001105A00E5
:1060500003105900012058000320560040A2E4F12B
:10606000646891060041A3E5F265699207000000AB
:1060700043414E464449666163653A204D657373FA
:106080006167652052414D204F766572666C6F776F
:10609000210000004261642043414E49666163650E
:1060A00020696E6465782E00000100000001FF0089
:1060B00000A0004000A4004000000000000000001C
:1060C000912C000869250008CD33000861250008DF
:1060D000D9250008E929000851270008A125000852
:1060E000A52500087D25000865250008A9290008C8
:1060F0008925000835350008952500087D29000808
:1061000000960000000000000000000000000000F9
:106110000000000000000000000000005D4C0008CE
:10612000494C0008854C0008714C00087D4C000863
:10613000694C0008554C0008414C0008914C00087F
:106140006330000040610008D86C0020E86E002039
:1061500000000020000002000200000000010030EA
:1061600000FF0300080000000000002400000800F9
:10617000040000000004000000FC00000200000019
:10618000000004300080000008000000000000381B
:1061900000000100010000006D61696E0069646C1F
:1061A000650000000000002800000000AAAAAAAABA
:1061B00000000024FFFF00000000000000000000BD
:1061C00000A0550A00000000AAAA9AAA00500000E8
:1061D000FFF20000000000770000990000000000BE
:1061E00000000000AAAAAAAA00000000FFFF000009
:1061F00000000000000000005A0000000000000045
:106200009AAAAAAA00000000F3FF0000990000006B
:10621000000000000A00000000000000AAAAAAAACC
:1062200005000000FFFF00008800000000000000E3
:106230000000000000000000AAAAAAAA00000000B6
:10624000FFFF000000000000000000000000000050
:1062500000000000AAAAAAAA00000000FFFF000098
:10626000000000000000000000000000000000002E
:10627000AAAAAAAA00000000FFFF00000000000078
:10628000000000000000000000000000AAAAAAAA66
:1062900000000000FFFF0000000000000000000000
:1062A0000000000000000000AAAAAAAA0000000046
:1062B000FFFF0000000000000000000000000000E0
:1062C00000000000AAAAAAAA00000000FFFF000028
:1062D000000000000000000048A0FF7F0100000057
:1062E000130400000000000000001800000000007F
:1062F000FE2A0100D2040000FF000000A463002079
:1063000010640020000000002060000883040000EA
:106310002B60000850040000396000084022002073
:10632000000000000000000000000000000000006D
:10633000000000000000000000000000000000005D
:10634000000000000000000000000000000000004D
:10635000000000000000000000000000000000003D
:10636000000000000000000000000000000000002D
:10637000000000000000000000000000000000001D
:00000001FF
